:1000000000000A128A111228FE00030EF1000408F3
:10001000F2000A08F300831203137F08F4000A16A3
:100020008A11C62B83010308A0000A128A11DE2F51
:10003600013400341C3083120313AF008830B00043
:100046000A128A11FB220A128A1142300A168A15EE
:100056009E240A128A1142300A168A1191240A1223
:100066008A11831203132808D1002708D000003014
:100076005102C83003195002031CBF280130510237
:100086004130031950020318BF285108CF00500809
:10009600CE00013083160313850001308316031743
:1000A60088008312031306158230C100DD30C000BC
:1000B600C00B5B28C10B5B28602800300A168A1526
:1000C60062270A128A11831203132208CD0021081F
:1000D600CC0006114C08AE004D08AF00B001B101CE
:1000E6004E08A1004F08A200A301A4010030A800F9
:1000F6000030A7000330A600E830A5000A168A11D2
:1001060083210A128A11831203132408B5002308D7
:10011600B4002208B3002108B2000A168A11EA25A3
:100126000A128A11831203132F08D3002E08D20055
:100136005308C0004008A10001300A168A1532276C
:100146000A128A11831203135208C0004008A10044
:1001560002300A168A1532270A128A11593083127A
:100166000313AF008A30B0005308B2005208B10042
:100176000A128A11FB220800403083120313AF00D3
:100186008E30B0000A128A11FB2208001E3083123C
:100196000313CF000030D0000730D1000030D2006A
:1001A6000A30D3000030D40006160730CD007D306B
:1001B600CC00CC0BDC28CD0BDC2883120313861570
:1001C600A730AF008E30B0000A128A11FB220A1245
:1001D6008A1183120313D501D60150085602031D56
:1001E600F6284F08550203181129640006308312B9
:1001F6000313CE001330CD00B130CC00CC0B012957
:10020600CD0B0129CE0B01290829013083120313D6
:10021600D5070318D60A0030D607F028061286112D
:100226008230CD00DD30CC00CC0B1729CD0B172941
:100236001C296E3083120313AF008D30B0000A12F2
:100246008A11FB220A128A110A168A1102250A123B
:100256008A11243083120313AF008D30B0000A12C6
:100266008A11FB220A128A110A168A1176250A12A7
:100276008A110A168A15E4240A128A112D3083126D
:100286000313AF008F30B0000A128A11FB220A1244
:100296008A1183120313D501D60152085602031D93
:1002A6005629510855020318712964000630831235
:1002B6000313CE001330CD00B130CC00CC0B612936
:1002C600CD0B6129CE0B61296829013083120313F6
:1002D600D5070318D60A0030D60750295130AF008B
:1002E6008F30B0000A128A11FB220A128A110A16EE
:1002F6008A1579250A128A1183120313D501D601AC
:1003060054085602031D8929530855020318A429C7
:100316006400063083120313CE001330CD00B130D3
:10032600CC00CC0B9429CD0B9429CE0B94299B2978
:10033600013083120313D5070318D60A0030D607F7
:1003460083290A168A15D8240A128A116E30831256
:100356000313AF008D30B0000A128A11FB220A1275
:100366008A110A168A1102250A128A111A30831274
:100376000313CD00F830CC00CC0BBF29CD0BBF2921
:100386000000243083120313AF008D30B0000A1230
:100396008A11FB220A128A110A168A11762508008A
:1003A600863083120313AF008D30B0000A128A1113
:1003B600FB220A128A11D53083120313AF008C3048
:1003C600B0000A128A11FB220A128A11ED3083123A
:1003D6000313AF008A30B0000A128A11FB220A12F8
:1003E6008A11C83083120313AF008A30B0000A1294
:1003F6008A11FB220A128A11EE3083120313AF0010
:100406008830B0000A128A11FB220A128A112F3094
:1004160083120313AF008C30B0000A128A11FB223C
:100426000A128A114B3083120313AF008C30B000CE
:100436000A128A11FB220A128A113430831203131C
:10044600AF008B30B0000A128A11FB220A128A1101
:100456002A3083120313AF008E30B0000A128A11BD
:10046600FB220A128A11FD3083120313AF008D306E
:10047600B0000A128A11FB220A128A11BA308312BC
:100486000313AF008C30B0000A128A11FB220A1245
:100496008A11C33083120313AF008830B0000A12EA
:1004A6008A11FB220A128A11973083120313AF00B6
:1004B6008B30B0000A128A11FB220A128A11A3306D
:1004C60083120313AF008A30B0000A128A11FB228E
:1004D6000A128A110D3083120313AF008A30B0005E
:1004E6000A128A11FB220A128A114430831203135C
:1004F600AF008930B0000A128A11FB220A128A1153
:10050600BE3083120313AF008930B0000A128A117D
:10051600FB220A128A11563083120313AF008B3066
:10052600B0000A128A11FB220A128A11963083122F
:100536000313AF008930B0000A128A11FB220A1297
:100546008A11E63083120313AF008930B0000A1215
:100556008A11FB220A128A11123083120313AF008A
:100566008B30B0000A128A11FB220A128A117730E8
:1005760083120313AF008B30B0000A128A11FB22DC
:100586000A128A11333083120313AF008A30B00087
:100596000A128A11FB220A128A11F53083120313FA
:1005A600AF008B30B0000A128A11FB220A128A11A0
:1005B600123083120313AF008C30B0000A128A1176
:1005C600FB220A128A11B73083120313AF008B3055
:1005D600B0000A128A11FB220A128A11D63083123F
:1005E6000313AF008B30B0000A128A11FB220800F9
:1005F600313083120313B5003508BC008312031390
:100606003008B6002F08B500AF0A0319B00A36083D
:10061600FF00350884000A128A1500200A128A1182
:10062600B7003708BF003F080319080025303F060A
:100636000319242B3F080A168A153A260A128A112C
:10064600012B83120313B901602B3C08840083132A
:100656000008BA00840A00088403BB000230B50013
:100666003508BC073A083B04031D3D2BCB30BA00C6
:100676009030BB003B08FF003A0884000A128A1536
:1006860000200A128A11003A0319012B3B08FF00C9
:100696003A0884000A128A1500200A128A110A16DC
:1006A6008A153A260A128A11013083120313BA07F1
:1006B6000318BB0A3D2B3917812B3008B6002F08CB
:1006C600B500AF0A0319B00A3608FF0035088400E2
:1006D6000A128A1500200A128A11BF00003A03196D
:1006E600262C643A0319812B0D3A0319812B1A3AE9
:1006F6000319282B063A03195E2B012B391B9B2B5A
:100706003C08840083130008BD00840A0008BE006C
:100716000230B5003508BC07BE1FA72B0330B50055
:100726003508B904BD09BE09BD0A0319BE0AA72BBF
:100736003C08840083130008BD00840A0008BE003C
:100746000230B5003508BC07BF01BF0A05303F06B9
:100756000319D22B3F08B5003507123E84008830B6
:100766000318013EFF000A128A1500200A128A1198
:10077600B6000A128A1500200A128A11B700370835
:100786003E02031DC82B36083D02031CD22B013046
:10079600B5003508BF0705303F06031DAD2B3908E8
:1007A60003390319DC2B2D300A168A153A260A124C
:1007B6008A11831203133F08B5003508B800FF30CD
:1007C60083120313B5003508B807380A0319012B3D
:1007D6000A30A9000030AA003808B5003507123ED5
:1007E600840088300318013EFF000A128A15002093
:1007F6000A128A11A1000A128A1500200A128A1109
:10080600A2003E08A4003D08A3000A168A1145214D
:100816000A128A11831203132208AC002108AB00C6
:100826000A168A1595270A128A11831203132908B4
:10083600303EB6003608BF003F080A168A153A262B
:100846000A128A11E22B0800031003178312201ED6
:10085600031400300318013083120313E10064000F
:100866001730831203178500F830831603138100AF
:10087600073085000730831603178800013083167A
:100886000313860083160317890183160313870152
:10089600831203138501860187018230D800DD307B
:1008A600D700D70B542CD80B542C592C8312031376
:1008B600DD018B130A168A1522250A128A110A16D9
:1008C6008A15F1240A128A110A168A15C3250A12F4
:1008D6008A110A168A15AE240A128A118B17E63077
:1008E60083120313AF008D30B0000A128A11FB2267
:1008F6000A128A1183160313E201E301F53083120B
:100906000313AF009030B0000A128A11FB220A12BC
:100916008A110A168A1578260A128A11031CD32C04
:100926000A168A1559260A128A1183120313D7004A
:10093600570883160313E30008306306031DB72C1C
:1009460062080319D32C0130E20263080A168A15DD
:100956003A260A128A1120300A168A153A260A12EF
:100966008A1183160313CD2C83160313630883128F
:100976000313D700831603136208D23E8400831242
:1009860003135708831380000130D70057088316D6
:100996000313E20763080A168A153A260A128A1111
:1009A6006400831203135B085C040319152D0A16F1
:1009B6008A159A260A128A11831203132108D70070
:1009C6002208D8005C08A2005B08A1003C30A30006
:1009D6000030A4000A168A15BC260A128A11831250
:1009E600031322085802031DFA2C21085702031C80
:1009F600152DD030AF008F30B0000A128A11FB22BD
:100A06000A128A110A168A113B270A128A11053020
:100A160083120313D7005708E10083160313E2017C
:100A2600E20A1F2D0D3083160313630603191F2DCB
:100A36000F306202031C8C2C6208FF3ED23E8400FB
:100A460083138001520803197D2C5230831203133D
:100A5600A1009030A200D2300A168A1503270A1286
:100A66008A118312031321082204031D402D0A163E
:100A76008A113B270A128A117D2C873083120313B1
:100A8600A1009030A200D2300A168A1503270A1256
:100A96008A118312031321082204031D582D0A16F6
:100AA6008A1163220A128A117D2CA2308312031343
:100AB600A1009030A200D2300A168A1503270A1226
:100AC6008A118312031321082204031D702D0A16AE
:100AD6008A11C4210A128A117D2C0730831203134E
:100AE600A1009030A200D2300A168A1503270A12F6
:100AF6008A118312031321082204031D882D0A1666
:100B06008A11B5220A128A117D2C4E3083120313E4
:100B1600A1009030A200D2300A168A1503270A12C5
:100B26008A118312031321082204031DA02D0A161D
:100B36008A15FE250A128A117D2C62308312031350
:100B4600A1009030A200D2300A168A1503270A1295
:100B56008A118312031321082204031DB82D0A16D5
:100B66008A15E0250A128A117D2CC43083120313DC
:100B7600A1008F30A200D2300A168A1503270A1266
:100B86008A118312031321082204031DD02D0A168D
:100B96008A151C260A128A117D2CAB308312031388
:100BA600A1009030A200D2300A168A1503270A1235
:100BB6008A118312031321082204031DE82D0A1645
:100BC6008A15E4240A128A117D2C753083120313C8
:100BD600A1009030A200D2300A168A1503270A1205
:100BE6008A118312031321082204031D002E0A16FC
:100BF6008A15D8240A128A117D2CEE30831203132B
:100C0600A1009030A200D2300A168A1503270A12D4
:100C16008A118312031321082204031D182E0A16B3
:100C26008A1590250A128A117D2CC330831203136C
:100C3600A1009030A200D2300A168A1503270A12A4
:100C46008A118312031321082204031D302E0A126F
:100C56008A111D200A128A117D2C993083120313E2
:100C6600A1009030A200D2300A168A1503270A1274
:100C76008A118312031321082204031D482E0A1623
:100C86008A1179260A128A117D2C303083120313B9
:100C9600A1009030A200D2300A168A1503270A1244
:100CA6008A118312031321082204031D602E0A16DB
:100CB6008A1102250A128A117D2C3A3083120313F7
:100CC600A1009030A200D2300A168A1503270A1214
:100CD6008A118312031321082204031D782E0A1693
:100CE6008A1176250A128A117D2CE63083120313A7
:100CF600A1008F30A200D2300A168A1503270A12E5
:100D06008A118312031321082204031D902E0A164A
:100D16008A110E210A128A117D2CFC3083120313CC
:100D2600A1008F30A200D2300A168A1503270A12B4
:100D36008A118312031321082204031DA82E0A1602
:100D46008A15CD240A128A117D2C263083120313AC
:100D5600A1009030A200D2300A168A1503270A1283
:100D66008A118312031321082204031DC02E0A16BA
:100D76008A15C2240A128A117D2CDB3083120313D2
:100D8600A1008F30A200D2300A168A1503270A1254
:100D96008A118312031321082204031DD82E0A1672
:100DA6008A15C9270A128A117D2CF1308312031382
:100DB600A1008F30A200D2300A168A1503270A1224
:100DC6008A118312031321082204031DF02E0A162A
:100DD6008A15B7240A128A117D2C58308312031300
:100DE600A1009030A200D2300A168A1503270A12F3
:100DF6008A118312031321082204031D082F0A16E1
:100E06008A1562250A128A117D2C903083120313EB
:100E1600A1009030A200D2300A168A1503270A12C2
:100E26008A118312031321082204031D202F0A1698
:100E36008A154B250A128A117D2CB83083120313AA
:100E4600A1008F30A200D2300A168A1503270A1293
:100E56008A118312031321082204031D382F0A1650
:100E66008A1579250A128A117D2C6C308312031398
:100E7600A1009030A200D2300A168A1503270A1262
:100E86008A118312031321082204031D502F0A1608
:100E96008A1108230A128A117D2C7E3083120313CD
:100EA600A1009030A200D2300A168A1503270A1232
:100EB6008A118312031321082204031D682F0A16C0
:100EC6008A1112220A128A117D2C443083120313CE
:100ED600A1009030A200D2300A168A1503270A1202
:100EE6008A118312031321082204031D802F0A1678
:100EF6008A15A9250A128A117D2C1C308312031328
:100F0600A1009030A200D2300A168A1503270A12D1
:100F16008A118312031321082204031D982F0A1233
:100F26008A11C9200A128A117D2CFA308312031302
:100F3600A1009030A200D2300A168A1503270A12A1
:100F46008A1183120313210822040319BA2F0B30C6
:100F5600A1009130A200D2300A168A1503270A1280
:100F66008A118312031321082204031DC02F0A12BB
:100F76008A11D3210A128A117D2CFF3083120313A2
:100F8600A1009030A200D2300A168A1503270A1251
:100F96008A118312031321082204031DD82F0A166F
:100FA6008A1536250A128A117D2C083083120313FE
:100FB600AF008F30772CF901F501F601F701F80142
:100FC600D901DA01DB01DC01DD01DE018313A0308A
:100FD6008400D2300A168A15A6240A128A110A1229
:100FE6008A111B200A128A11DF000A128A111C209C
:100FF600E00083010A128A11272CFF1B0A2883139B
:101006007F1883170008840A0319FF0A08007F085F
:101016007F398A000408840A0319FF0A8200013412
:1010260000340A34003464340034E83403341034B1
:1010360027340D340A3445346E34743465347234CE
:101046002034613463347434753461346C34203440
:1010560069346E34703475347434203476346F34B5
:101066006C347434613467346534203469346E34D6
:101076002034643465346334693476346F346C34C4
:1010860074347334203428343234303430342034D9
:101096002D3420343334323430342C34203430344C
:1010A600203474346F342034613462346F347234D3
:1010B600743429343A34203400340D340A34453437
:1010C6006E347434653472342034743469346D3457
:1010D60065346F3475347434203469346E34203496
:1010E6006D3469346E347534743465347334203435
:1010F6002834313420342D342034313430343934EA
:1011060032342C3420343034203466346F34723424
:1011160020346E34653476346534723429343A3486
:10112600203400340D340A3445346E347434653456
:1011360072342034733465347234693461346C34F7
:1011460020346E3475346D34623465347234203430
:101156002834313420342D34203432343534353487
:101166002C3420343034203474346F3420346134D9
:1011760062346F347234743429343A34203400348F
:1011860073346534743462346134743474340934B9
:1011960009347334653474342034623461347434FD
:1011A6007434653472347934203476346F346C3464
:1011B60074346134673465342034633461346C3498
:1011C6006934623472346134743469346F346E3421
:1011D6000D340A3400347334653474347434693429
:1011E6006D3465346F34753474340934733465344E
:1011F600743420346D346134783420347434693472
:101206006D34653420346134773461346B3465343D
:10121600203469346E3420346D3469346E34753458
:101226007434653473340D340A3400340D340A349E
:1012360045346E34743465347234203473346C340B
:101246006534653470342034743469346D346534EF
:10125600203469346E3420346D3469346E34753418
:1012660074346534733420342834313420342D34C6
:101276002034313430343934323429343A34203459
:1012860000346334683467347234733474347234BB
:101296006F346234653409346334683461347234CB
:1012A600673465342034723469346734683474348E
:1012B60020347334743472346F34623465342034B9
:1012C60076346F346C3474346134673465340D3479
:1012D6000A3400340D340A3445346E3474346534BB
:1012E60072342034643465346C3461347934203497
:1012F600743469346D346534203469346E34203482
:101306007334653463346F346E3464347334203428
:101316002834303420342D342034363430342934D3
:101326003A34203400346334683467346C347334AC
:10133600743472346F346234653409346334683417
:10134600613472346734653420346C346534663401
:10135600743420347334743472346F3462346534C4
:10136600203476346F346C347434613467346534C5
:101376000D340A34003472347334743472346F3476
:10138600623465346F34663466340934203472341A
:101396006934673468347434203473347434723482
:1013A6006F346234653420346334683461347234A3
:1013B600673469346E34673420346F346634663487
:1013C6000D340A3400346C347334743472346F342C
:1013D600623465346F3466346634093420346C34D0
:1013E60065346634743420347334743472346F3430
:1013F600623465342034633468346134723467345B
:1014060069346E34673420346F34663466340D3490
:101416000A34003472346534613464347234763498
:101426006D346F346E340934723465346134643427
:101436002034723469346734683474342034733435
:10144600743472346F3462346534203476346F34D5
:101456006C3474346134673465340D340A340034C2
:10146600743472346934673473346834753474345C
:101476007434653472340934203474347234693403
:1014860067346734653472342034633461346D34C0
:10149600653472346134203473346834753474348A
:1014A6007434653472340D340A3400340D340A341D
:1014B6004734613469346E342034763461346C34A4
:1014C6007534653420346F346634203425347534ED
:1014D600203473346134763465346434203474349F
:1014E6006F34203445344534503452344F344D34FF
:1014F6000D340A3400340D340A34533465347234EE
:10150600693461346C3420346E3475346D3462342D
:1015160065347234203425347534203473346134A0
:10152600763465346434203474346F34203445346E
:101536004534503452344F344D340D340A3400346B
:1015460072346534613464346C3476346D346F349B
:101556006E340934723465346134643420346C3446
:1015660065346634743420347334743472346F34AE
:1015760062346534203476346F346C3474346134B8
:10158600673465340D340A34003473346534743486
:10159600643465346C3461347934093473346534B5
:1015A60074342034643465346C34613479342034D2
:1015B600743469346D346534203469346E342034BF
:1015C6007334653463346F346E34643473340D3479
:1015D6000A34003473346534743473346C346534CB
:1015E6006534703409347334653474342034733498
:1015F6006C346534653470342034743469346D3435
:101606006534203469346E3420346D3469346E3474
:1016160075347434653473340D340A3400347434D8
:1016260072346934673472346934673468347434B4
:101636000934203474347234693467346734653459
:101646007234203472346934673468347434203424
:101656007334743472346F34623465340D340A343E
:1016660000347234653461346434743469346D34EE
:1016760065346F34753474340934723465346134C6
:10168600643420346D3461347834203474346934ED
:101696006D34653420346134773461346B346534A9
:1016A6000D340A3400346C347334743472346F3449
:1016B600623465346F346E340934203474347534CE
:1016C60072346E3420346C346534663474342034A9
:1016D6007334743472346F346234653420346F3446
:1016E6006E340D340A340034743472346934673419
:1016F6006C3465346634743409342034743472348A
:101706006934673467346534723420346C34653434
:101716006634743420347334743472346F346234FF
:1017260065340D340A3400347234653461346434FB
:101736006234613474347434093472346534613417
:1017460064342034623461347434743465347234ED
:101756007934203476346F346C34743461346734BD
:1017660065340D340A3400347234653461346434BB
:101776007334653472346E346F34093472346534BC
:1017860061346434203473346534723469346134BA
:101796006C3420346E3475346D346234653472348E
:1017A6000D340A340034683465346C3470342034B3
:1017B6006F34723420343F340934703472346934EF
:1017C6006E347434203463346F346D346D34613464
:1017D6006E34643420346C346934733474340D34A8
:1017E6000A340034743461346B34653469346D34CE
:1017F60061346734653409342034743461346B34AD
:101806006534203474346534733474342034693464
:101816006D346134673465340D340A3400347334FE
:10182600653474347334653472346E346F34093409
:1018360073346534743420347334653472346934E3
:1018460061346C3420346E3475346D3462346534EE
:1018560072340D340A3400347234653461346434BD
:1018660073346C34653465347034093472346534D9
:1018760061346434203473346C34653465347034C4
:101886002034743469346D3465340D340A340034CC
:101896007234653461346434643465346C34613470
:1018A60079340934723465346134643420346434F0
:1018B60065346C34613479342034743469346D346D
:1018C60065340D340A3400340D340A3453346C3420
:1018D6006534653470342034743469346D34653459
:1018E6002034733465347434203474346F342034C3
:1018F600253464342034253473340D340A340034EA
:101906000D340A34443465346C346134793420340B
:10191600743469346D346534203473346534743406
:10192600203474346F342034253464342034253420
:1019360073340D340A3400340D340A3449346E34A9
:10194600763461346C3469346434203473346534E9
:101956007234693461346C3420346E3475346D34C9
:1019660062346534723421340D340A3400347234EE
:101976006534613464343734763409340934723466
:1019860065346134643420347334743461347434AB
:10199600653420346F3466342034373456340D348D
:1019A6000A34003473346C34653465347034093465
:1019B600093473346C3465346534703420346134DE
:1019C60066347434653472342034643465346C346B
:1019D600613479340D340A3400340D340A34523407
:1019E600693467346834743420345334743472344C
:1019F6006F34623465342034543472346934673455
:101A060067346534723420340D340A3400340D34AE
:101A16000A345234693467346834743420345334A5
:101A2600743472346F346234653420344334683429
:101A360061347234673469346E3467340D340A3471
:101A460000340D34523469346734683474342034C5
:101A56005334743472346F346234653420345634FB
:101A66006F346C3474346134673465343A340D340D
:101A76000A3400340D340A34543469346D34653410
:101A86006F347534743420347334653474342034CC
:101A960074346F342034253464342034253473345C
:101AA6000D340A3400340D344C34653466347434E1
:101AB60020345334743472346F34623465342034D1
:101AC600543472346934673467346534723420347C
:101AD6000D340A3400340D344C34653466347434B1
:101AE60020345334743472346F34623465342034A1
:101AF60056346F346C3474346134673465343A3434
:101B06000D340A3400340D340A34563461346C34DE
:101B160069346434203463346F346D346D34613425
:101B26006E346434733420346134723465343A3438
:101B36000D340A3400340D344C3465346634743450
:101B460020345334743472346F3462346534203440
:101B56004334683461347234673469346E346734BC
:101B66000D340A3400340D340A3453346C3465347D
:101B7600653470342034743469346D3465342034FB
:101B86006934733420342534753420342534733461
:101B96000D340A3400340D340A34443465346C345C
:101BA600613479342034743469346D3465342034C6
:101BB6006934733420342534753420342534733431
:101BC6000D340A3400340D340A3452346F3476340A
:101BD600653472342034573461346B346534793467
:101BE6002034763431342E3433342E3430340D34BC
:101BF6000A340034733465347434373476346F34CD
:101C06006634663409347434753472346E34203470
:101C16003734563420346F34663466340D340A341F
:101C260000340D340A3453346C34653465347034FE
:101C360069346E34673420342534753420342534C1
:101C460073342E342E342E340D340A340034733467
:101C560065347434373476346F346E340934093469
:101C66007434753472346E34203437345634203438
:101C76006F346E340D340A3400340D340A3449346A
:101C86006E34763461346C3469346434203476349A
:101C96006F346C34743461346734653421340D34F4
:101CA6000A3400340D340A345234693467346834E3
:101CB600743420345334743472346F34623465347B
:101CC60020344F34663466340D340A3400340D340F
:101CD6000A34543469346D3465346F34753474346D
:101CE6002034693473342034253475342034253453
:101CF60073340D340A3400340D3454347234693478
:101D06006734673465347234203453346834753438
:101D1600743474346534723420340D340A34003427
:101D26000D340A344C3465346634743420345334F8
:101D3600743472346F346234653420344F3466340C
:101D460066340D340A3400340D345334743472342A
:101D56006F34623465347334203443346834613408
:101D66007234673469346E3467340D340A3400349F
:101D76000D340A347734613474346334683464342B
:101D86006F3467342034773461346B34653475349A
:101D960070340D340A3400340D340A344C3465344E
:101DA6006634743420345334743472346F34623489
:101DB600653420344F346E340D340A3400340D3417
:101DC6000A34743469346D3465346F34753474345C
:101DD6002034773461346B346534753470340D34A3
:101DE6000A3400340D340A3477346134743463347D
:101DF600683464346F346734203472346534733431
:101E0600653474340D340A3400340D340A344934DC
:101E16006E34763461346C3469346434203463341B
:101E26006F346D346D3461346E346434213400346F
:101E36000D340A3449346E34763461346C34693482
:101E460064342034743469346D34653421340D348B
:101E56000A3400340D345434753472346E342034FC
:101E66004F346E342034433461346D346534723407
:101E760061340D340A3400340D340A346E346F3450
:101E860072346D3461346C342034773461346B349D
:101E96006534753470340D340A3400340D344334EB
:101EA6006134703474347534723465342034493492
:101EB6006D346134673465340D340A3400340D34BE
:101EC6000A346D346F34643465346D3420347734B9
:101ED60061346B346534753470340D340A3400342F
:101EE6000D340A346E346F3472346D3461346C34AC
:101EF6002034723465347334653474340D340A34E2
:101F060000340D340A34373456342034693473348B
:101F160020344F34463446340D340A3400340D34FC
:101F26000A343734563420346934733420344F3409
:101F36004E340D340A3400340D340A3437345634F2
:101F46002034693473342034253473340D340A3420
:101F560000340D340A3475346E346B346E346F3499
:101F660077346E340D340A34003474347234693480
:101F76006734733468347534743474346534723445
:101F860000347234653461346434743469346D34C5
:101F960065346F347534743400340D340A34543473
:101FA60069346D3465346F347534743421340034D7
:101FB6006334683467346C347334743472346F3415
:101FC600623465340034633468346734723473348D
:101FD600743472346F346234653400346C34733460
:101FE600743472346F34623465346F3466346634F4
:101FF600003472347334743472346F34623465343A
:102006006F3466346634003473346534743474342F
:1020160069346D3465346F347534743400340D347A
:102026000A34253475342E34253475340D340A3487
:102036000034743461346B34653469346D3461341E
:102046006734653400346C347334743472346F34EA
:10205600623465346F346E340034723465346134FE
:1020660064346C3476346D346F346E3400347234C8
:10207600653461346434723476346D346F346E345E
:1020860000347234653461346434733465347234C4
:102096006E346F34003472346534613464347334AE
:1020A6006C34653465347034003474347234693495
:1020B6006734723469346734683474340034723483
:1020C600653461346434643465346C346134793431
:1020D60000347234653461346434773461346B347B
:1020E60065340034733465347434373476346F347D
:1020F600663466340034733465347434733465344A
:1021060072346E346F34003473346534743473341B
:102116006C34653465347034003474347234693424
:1021260067346C3465346634743400347234653420
:102136006134643462346134743474340034733416
:1021460065347434643465346C3461347934003401
:10215600733465347434373476346F346E34003403
:102166007334653463346F346E34643473340034DA
:102176006D3469346E3475347434653473340034B4
:1021860073346534743462346134743474340034B2
:1021960028346E3475346C346C34293400340D3480
:1021A6000A34253475340D340A3400344134773416
:1021B60061346B34653421340034733465346334EC
:1021C6006F346E34643400346D3469346E3475346F
:1021D60074346534003472346534613464343734AD
:1021E600763400340D340A343E34203400346834F6
:1021F60065346C3470340034743465347334743438
:1022060000344F344634463400344F344E340034B0
:042216003F3400341D
:10221C00383083120313C3000030C40086150A3013
:10222C00AF008D30B0000A128A11FB220A168A11F7
:10223C0083120313C501C60144084602031D282955
:10224C004308450203184329640006308312031324
:10225C00C2001330C100B130C000C00B3329C10B18
:10226C003329C20B33293A29013083120313C507D2
:10227C000318C60A0030C6072229861108008312EB
:10228C000313A701A8012108220403197E29A60122
:10229C00A60AA21B5D2901300310A10DA20DFF3E61
:1022AC00031D52290130A5002508A6074F2901302E
:1022BC000310A70DA80DFF3E031D5E292208240262
:1022CC00031D6A2921082302031C73292108A30278
:1022DC002208031CA403A402271401300310A20C2F
:1022EC00A10CFF3E031D74290130A602031D5D29BC
:1022FC002808A2002708A10008000030831203134D
:10230C00AD000030AC000030AB000030AA00211C46
:10231C00A3292508AA07260803110318013E031D4B
:10232C00AB07270803110318013E031DAC0728084F
:10233C0003110318013E031DAD070130A900031062
:10234C00A50DA60DA70DA80DA90BA52901300310ED
:10235C00A40CA30CA20CA10CFF3E031DAD29240858
:10236C00230422042104031D8D292D08A4002C080C
:10237C00A3002B08A2002A08A10008006D308312CC
:10238C000313AF008930B0000A128A11FB220A161F
:10239C008A1140300A168A159E240A168A1140307A
:1023AC000A168A1191240A168A118312031328081B
:1023BC00CD002708CC0000304D023D3003194C02F3
:1023CC000318082A4D08DA004C08D90059035A049E
:1023DC000319F429B330CA009030F729E030CA0051
:1023EC009030CB008330AF008C30B0005A08B20074
:1023FC005908B1004A08B3004B08B4000A128A11FC
:10240C00FB2208001B3083120313AF008F30B00087
:10241C000A128A11FB220800953083120313AF00B5
:10242C008830B0000A128A11FB220A168A11423037
:10243C000A168A159E240A168A1142300A168A1127
:10244C0091240A168A11831203132808CE00270838
:10245C00CD004D084E040319592A01304E020030AC
:10246C0003194D020318592A4D08C0004008CC002E
:10247C004C08C0004008A10000300A168A1532270B
:10248C000A168A117E3083120313AF008A30B00013
:10249C004C08C000C1014008B1004108B2000A124A
:1024AC008A11FB2208009F3083120313AF008C307B
:1024BC00B0000A128A11FB22080019308312031390
:1024CC00AF008930B0000A128A11FB220A168A1159
:1024DC0040300A168A159E240A168A1140300A16B4
:1024EC008A1191240A168A11831203132808CD002D
:1024FC002708CC004C084D040319AB2A04304D02BC
:10250C00453003194C020318AB2A4D08E0004C0867
:10251C00DF005F0360040319972ABB30CA009030B8
:10252C009A2AE730CA009030CB006730AF008C306D
:10253C00B0006008B2005F08B1004A08B3004B0855
:10254C00B4000A128A11FB2208001B3083120313F9
:10255C00AF008F30B0000A128A11FB2208006030E5
:10256C0083120313AF008830B0000A128A11FB22C9
:10257C000A168A1140300A168A159E240A168A11E8
:10258C0040300A168A1191240A168A1183120313F9
:10259C002808CD002708CC0004304D024530031923
:1025AC004C020318FE2A4D08DC004C08DB005B03D0
:1025BC005C040319E52ABB30CA009030E82AE730E6
:1025CC00CA009030CB003D30AF008D30B0005C08BD
:1025DC00B2005B08B1004A08B3004B08B4000A1201
:1025EC008A11FB220A168A110A168A15222508005E
:1025FC001B3083120313AF008F30B0000A128A1104
:10260C00FB2208004F2B733083120313AF008F3063
:10261C00B0000A128A11FB220800F5308312031352
:10262C00AF008E30B0000A128A11FB2208003F3036
:10263C0083120313AF008F30B0000A128A11FB22F1
:10264C000800BB3083120313AF008E30B0000A12A7
:10265C008A11FB220800623083120313AF008F3003
:10266C00B0000A128A11FB220800E2308312031315
:10267C00AF008E30B0000A128A11FB220800AC3079
:10268C0083120313AF008F30B0000A128A11FB22A1
:10269C000800831203136108003A0319092B013A4D
:1026AC000319132B033A03191D2B013A0319272B7A
:1026BC00073A0319312B013A03193B2B452B080020
:1026CC00003083120313BA000030B9000030B80098
:1026DC000030B700310830042F042E040319BD2B31
:1026EC00BB01BB0AB11B882B0130B6000310AE0D29
:1026FC00AF0DB00DB10DB60B7C2B0130B60036080A
:10270C00BB07782B0130B6000310B70DB80DB90D0F
:10271C00BA0DB60B8A2B31083502031D9F2B3008DE
:10272C003402031D9F2B2F083302031D9F2B2E08F1
:10273C003202031CB02B2E08B2022F08031C2F0FE1
:10274C00B3023008031C300FB4023108031C310FE4
:10275C00B502371401300310B10CB00CAF0CAE0C39
:10276C00FF3E031DB12B0130BB02031D882B3A0821
:10277C00B1003908B0003808AF003708AE000800C7
:10278C008C1EE42B831603138C1EE42B8312031371
:10279C001A08F0007508B03E84007008831380009E
:1027AC007508013E0F39F0007008DE005E087606F1
:1027BC000319E42B5E08F0007008F50083120C1E60
:1027CC00022C831603130C1E022C7808C03E8400C6
:1027DC00831300088312031399000130F000700872
:1027EC00F8070F30F0007008F80578087706031D1D
:1027FC00022C831603130C12831603130C1C1B2CB4
:10280C00831203130C1C1B2C101080308F00003013
:10281C008E001014013083160313D0070318D10A4D
:10282C000030D107831203130C1074088312FF00BD
:10283C0073088A0072088400710E8300FE0E7E0EEF
:10284C00090083120313AB002B08A7002708AC0068
:10285C00702C2B082C060319702C20300A168A15A4
:10286C003A260A168A1108300A168A153A260A16CA
:10287C008A11013083120313AC02702C08300A1633
:10288C008A153A260A168A1120300A168A153A2613
:10289C000A168A1108300A168A153A260A168A115F
:1028AC00013083120313AC022C082B020318702C7A
:1028BC00442C2C088400831380012B080800290861
:1028CC00A7002C0884002708831380000130A70080
:1028DC002708AC070A168A1510250A168A118312C6
:1028EC000313A700A8012708A9002808AA002A0892
:1028FC00003A0319822C652C2908083A03192F2C4D
:10290C00023A03195F2C073A03195F2C183A031982
:10291C005A2C652C702C83120313AE002E088400E5
:10292C00203083130006031DA02C0130A9002908B8
:10293C00AE07942C2E0884000930000603199B2C3A
:10294C00AC01AD01AB012E0884002D300006031D37
:10295C00B42C0130A9002908AB07BA2C2E0884002E
:10296C002B300006031DBE2C0130A9002908AE0730
:10297C002E08840000080A168A1500250A168A11EA
:10298C00031CEC2C831203132D08A2002C08A100AD
:10299C000A30A3000030A4000A168A15BC260A16B9
:1029AC008A11831203132E08840083130008210755
:1029BC00A90022080318220AAA002908D03EAC005C
:1029CC002A080318013EFF3EAD00BA2C83120313F4
:1029DC002B080319FD2C2C09A9002D09AA00A90A02
:1029EC000319AA0A2908A7002A08A80008002D081C
:1029FC00A8002C08A7000800003083120313C7009E
:102A0C000030C6000030C5003030C40007308316DB
:102A1C0003138500073083160317880001300A164C
:102A2C008A1562270A168A11831203132208C90019
:102A3C002108C8000030B1000030B0000030AF00F9
:102A4C006430AE003230C0000030C1000030C20033
:102A5C000030C3004808A1004908A200A301A4014A
:102A6C004708A8004608A7004508A6004408A5008A
:102A7C000A168A1183210A168A118312031321085C
:102A8C00C00722080318220F4C2D4D2DC107230817
:102A9C000318230F522D532DC20724080318240AA0
:102AAC00C3074308B5004208B4004108B30040080E
:102ABC00B2000A168A1166230A168A1183120313AE
:102ACC002F08CB002E08CA00D230AF009030B000D7
:102ADC004B08B2004A08B1000A128A11FB22080006
:102AEC00003083120313C7000030C6000030C5004D
:102AFC003030C4000730831603138500073083166B
:102B0C000317880002300A168A1562270A168A11E2
:102B1C00831203132208C9002108C8000030B10039
:102B2C000030B0000030AF006430AE003230C00076
:102B3C000030C1000030C2000030C3004808A100C2
:102B4C004908A200A301A4014708A8004608A70051
:102B5C004508A6004408A5000A168A1183210A1606
:102B6C008A11831203132108C00722080318220FAD
:102B7C00C02DC12DC10723080318230FC62DC72D47
:102B8C00C20724080318240AC3074308B5004208E7
:102B9C00B4004108B3004008B2000A168A1166233B
:102BAC000A168A11831203132F08CB002E08CA00B1
:102BBC00D230AF009030B0004B08B2004A08B100E0
:102BCC000A128A11FB22080083120313B801B11FE9
:102BDC00FC2DAE09AF09B009B109AE0A0319AF0A51
:102BEC000319B00A0319B10AB801B80AB51F0D2EA2
:102BFC00B209B309B409B509B20A0319B30A031926
:102C0C00B40A0319B50A0130B6003608B80600300C
:102C1C00BC000030BB000030BA000030B9003108F5
:102C2C0030042F042E040319622EB701B70AB11B0E
:102C3C002D2E0130B6000310AE0DAF0DB00DB10D41
:102C4C00B60B212E0130B6003608B7071D2E013009
:102C5C00B6000310B90DBA0DBB0DBC0DB60B2F2E63
:102C6C0031083502031D442E30083402031D442E56
:102C7C002F083302031D442E2E083202031C552E3E
:102C8C002E08B2022F08031C2F0FB3023008031CAE
:102C9C00300FB4023108031C310FB5023914013066
:102CAC000310B10CB00CAF0CAE0CFF3E031D562E36
:102CBC000130B702031D2D2E38080319702EB909E7
:102CCC00BA09BB09BC09B90A0319BA0A0319BB0A28
:102CDC000319BC0A3C08B1003B08B0003A08AF002D
:102CEC003908AE00080001300A168A15DF260A16CC
:102CFC008A1183120313C000C1014008C100C00136
:102D0C0002300A168A15DF260A168A11831203135B
:102D1C004007C4000030031801304107C500C6014C
:102D2C00C51BC6034608C700013083160313850074
:102D3C0001308316031788008312031306158230A3
:102D4C00C100DD30C000C00BA92EC10BA92EAE2EC8
:102D5C0000300A168A1562270A168A118312031389
:102D6C002208C9002108C80006110030B10000304B
:102D7C00B0000330AF00E830AE00F430C0000130DA
:102D8C00C1000030C2000030C3004808A10049084F
:102D9C00A200A301A4014708A8004608A700450803
:102DAC00A6004408A5000A168A1183210A168A1166
:102DBC00831203132108C00722080318220FE72EE1
:102DCC00E82EC10723080318230FED2EEE2EC207A1
:102DDC0024080318240AC3074308B5004208B400AA
:102DEC004108B3004008B2000A168A1166230A167D
:102DFC008A11831203132F08CF002E08CE000A303D
:102E0C00A1000030A2004F08A4004E08A3000A162F
:102E1C008A1145210A168A11831203132208CB004A
:102E2C002108CA000A30A9000030AA004F08AC00E3
:102E3C004E08AB000A168A1595270A168A118312BA
:102E4C0003132A08CD002908CC001230AF009030B3
:102E5C00B0004B08B2004A08B1004D08B4004C0851
:102E6C00B3000A128A11FB220800831203136008B4
:102E7C00A2005F08A1003C30A3000030A4000A1699
:102E8C008A15BC260A168A11831203132208C40061
:102E9C002108C3005F0360040319582FBB30C50021
:102EAC0090305B2FE730C5009030C6001430AF0077
:102EBC008E30B0006008B2005F08B1004508B30066
:102ECC004608B4000A128A11FB220A168A118312D0
:102EDC000313C701C8015A084802031D772F59086C
:102EEC0047020318922F6400063083120313C200AA
:102EFC001330C100B130C000C00B822FC10B822F28
:102F0C00C20B822F892F013083120313C7070318BA
:102F1C00C80A0030C807712F83160313981C922F10
:102F2C008C128312031398138501860104308700D9
:102F3C008316031301138B1083120313DD0110107E
:102F4C0080308F0000308E001014831603130C1485
:102F5C000B178B13BB2F63008312031310108030DD
:102F6C008F0000308E0010140C1083124808C10022
:102F7C004708C000C70A0319C80A41084402031DC8
:102F8C00C92F4008430203188B18CE2F031AB12FF8
:102F9C000A168A1522250A168A118B178B1CDA2F12
:102FAC00043083120313E52F83120313831D031EB6
:102FBC00E12F0230E52F831D031AE82F0330C000E8
:102FCC004008E1008230C100DD30C000C00BEC2FA6
:102FDC00C10BEC2FF12F0A168A15C3250A168A117C
:102FEC00D93083120313AF009030B0000A128A114B
:042FFC00FB220800AC
:10393C0083120313AD002D080A168A1127240800E0
:10394C0064008001840A0406031900340406A72CC1
:10395C004030831203139F008030831603139F00A3
:10396C0008008312031306129330AF008E30B000A0
:10397C000A128A11FB220800831203130616CF3099
:10398C00AF008E30B0000A128A11FB22080083129D
:10399C00031386115530AF008E30B0000A128A1115
:1039AC00FB220800831203138610DD018430AF0064
:1039BC008F30B0000A128A11FB2208008312031305
:1039CC008614DD01DD0A9230AF008F30B0000A1290
:1039DC008A11FB2208000F30831203139000101081
:1039EC0080308F0000308E001014831603130C14DB
:1039FC000B17080083120313A200A1013A30220214
:103A0C0003180E2D30302202031C0E2DA101A10A29
:103A1C00210C08000A168A1559260A168A158312D3
:103A2C000313A5002508A60026080A168A153A26AF
:103A3C0083120313260808007910831603130C183D
:103A4C007914831603130C10D001D101791C322D7B
:103A5C00831603130C140800831603130C100800B0
:103A6C00D23083120313AF009030B0000A168A15BF
:103A7C009A260A168A15831203132208B20021080B
:103A8C00B1000A128A11FB220800831203130516D7
:103A9C004130C100EE30C000C00B522DC10B522D75
:103AAC0000008312031305125630AF008D30B000A6
:103ABC000A128A11FB220800831203138515413068
:103ACC00C100EE30C000C00B692DC10B692D000088
:103ADC00831203138511F030AF008C30B0000A1242
:103AEC008A11FB2208008312031386168230C10050
:103AFC00DD30C000C00B802DC10B802D852D8312B5
:103B0C00031386127F30AF008E30B0000A128A1178
:103B1C00FB220800831203135D08031D992D04304A
:103B2C00C00091309C2D0830C0009130C1009F30F6
:103B3C00AF008F30B0004008B1004108B2000A124B
:103B4C008A11FB22080000300A168A15DF260A1695
:103B5C008A1583120313C0004008C200D230AF0094
:103B6C009030B0004208C000C1014008B1004108CB
:103B7C00B2000A128A11FB220800193083160313B3
:103B8C009900181518128312031398171816981207
:103B9C00831603130C128C161813831203131813A9
:103BAC0083160313981298160B17F801F701F601F8
:103BBC00F50108008312031359035A040319EA2D63
:103BCC00B330C0009030ED2DE030C0009030C1001B
:103BDC00CE30AF008D30B0005A08B2005908B10099
:103BEC004008B3004108B4000A128A11FB220800F5
:103BFC00831203135F0360040319082EBB30C0004B
:103C0C0090300B2EE730C0009030C100B630AF00C2
:103C1C008D30B0006008B2005F08B1004008B300FE
:103C2C004108B4000A128A11FB2208008312031304
:103C3C005B035C040319262EBB30C0009030292E88
:103C4C00E730C0009030C1006A30AF008E30B00059
:103C5C005C08B2005B08B1004008B3004108B40036
:103C6C000A128A11FB22080083120313A2007708A0
:103C7C00013E0F39780603193D2E8B138312031363
:103C8C002208A1007708C03E84002108831380001D
:103C9C007708013E0F39A1002108F70083160313A2
:103CAC000C168B1708000A168A1578260A168A1520
:103CBC000318622E6400592E8B137608B03E8400D4
:103CCC008313000883120313A3002308A4000130FC
:103CDC00A3002308F6070F30A3002308F6058B1763
:103CEC002408080083120313981C862E83160313D2
:103CFC009812981683120313181218160310080042
:103D0C00181D922E1A08A1002108A2008316031375
:103D1C00981298160310080075087606031D982E45
:103D2C000310080003140800F910831603130C1871
:103D3C00F914831603130C10510883120313A400F7
:103D4C0083160313500883120313A300F91CB22E1D
:103D5C00831603130C14B52E831603130C10831245
:103D6C0003132408A2002308A100080083120313E4
:103D7C00A501A601211CC82E2308A5070318A60A15
:103D8C002408A60701300310A30DA40DFF3E031D4C
:103D9C00C92E01300310A20CA10CFF3E031DD02E26
:103DAC0021082204031DC02E2608A2002508A1000C
:103DBC00080083120313A200E52E83120313640080
:103DCC00831603178C18E32E831203132208831215
:103DDC0003178D003F3083120313A10021088316B3
:103DEC0003178C050C1403100C1803140030031863
:103DFC000130831203170C08080083120313A6006A
:103E0C000F2F0130A3002308A6070130A1070318C8
:103E1C00A20A2608840083130008A3002208FF00CE
:103E2C00210884000A128A1500200A168A15FF3A06
:103E3C00013E2307A4002408A5002508031D2C2FF0
:103E4C002608840083130008031D072F2508A100F2
:103E5C00A201A11BA203080083120313A300831663
:103E6C0003178C18352F831203132308831203179F
:103E7C008D00831203132108831203178C003F302B
:103E8C0083120313A2002208831603178C058312D6
:103E9C00031303108B1B03148B13831603170C15BE
:103EAC0055308D00AA308D008C140C118312031325
:103EBC00031C08008B17080083120313A7000F3094
:103ECC00A3002308A705C330A30023089F052708D8
:103EDC00A30001300310A30DFF3E031D702F031030
:103EEC00230DA40024089F041F14F930A300000024
:103EFC00A30B7D2F812F0000831203139F149F1897
:103F0C00852F1E08A600831603131E0883120313A5
:103F1C00A5001F102608A2002508A1000800831286
:103F2C00031329082A040319C42FAE01AE0AAA1BD5
:103F3C00AB2F01300310A90DAA0DFF3E031DA02FBE
:103F4C000130AD002D08AE079D2F2A082C02031D51
:103F5C00B12F29082B02031CB92F2908AB022A0800
:103F6C00031CAC03AC0201300310AA0CA90CFF3EDD
:103F7C00031DBA2F0130AE02031DAB2F2C08AA0073
:103F8C002B08A9000800343083120313C30000303F
:103F9C00C40006169E30AF008D30B0000A128A1194
:103FAC00FB220A168A1583120313C501C6014408A5
:103FBC004602031DE32F430845020318FE2F64003D
:103FCC00063083120313C2001330C100B130C0009D
:103FDC00C00BEE2FC10BEE2FC20BEE2FF52F0130C5
:103FEC0083120313C5070318C60A0030C607DD2F5A
:043FFC0006120800A1
:02400E00DAECEA
:00000001FF
